S31508001800000A0020D9180008E7180008E918000897
S3150800181000000000000000000000000000000000BA
S315080018200000000000000000000000000119000888
S31508001830000000000000000003190008C137000876
S31508001840CD420008071900080719000807190008FB
S3150800185007190008071900080719000807190008DA
S31508001860071900089528000807190008071900082D
S3150800187007190008071900080719000807190008BA
S3150800188007190008000000000000000007190008FA
S3150800189000000000071900080719000807190008C2
S315080018A0000000000719000807190008ED3C0008A9
S315080018B007190008071900080719000800000000A2
S315080018C0EE11AA550348854600F0B2FC00480047C9
S315080018D085500008000A00200B4880F308880B484A
S315080018E080470B480047FEE704207146084202D0AD
S315080018F0EFF3098001E0EFF30880714603F0C0FAC0
S31508001900FEE7FEE7FEE7FEE7000A00203D3900088D
S31508001910C518000830B50B460146002020220124D0
S3150800192009E00D46D5409D4205D31D469540491B05
S315080019302546954040191546521E002DF1DC30BD4E
S3150800194070B500242546002801DA01244042002902
S3150800195001DA01254942FFF7DDFFAC4200D04042DB
S31508001960002C00D0494270BD03460B439B0703D0A9
S3150800197009E008C9121F08C0042AFAD203E00B7846
S315080019800370401C491C521EF9D27047D2B201E0BE
S315080019900270401C491EFBD270470022F6E710B5BC
S315080019A013460A4604461946FFF7F0FF204610BDBF
S315080019B0F8B502464A40D40F42004B0052085B086D
S315080019C09A4202D20246084611464A0023D0C30D5F
S315080019D04A00DDB2120EAD1A202D35DA490201266B
S315080019E0490AF6058A19002C00D0524220214F1BBD
S315080019F01146B9402A411018C20D9A4221D0002C2E
S31508001A0017D0012D08DCDA05801AD20F8019D20703
S31508001A10DBB200F023FBF8BDDA05801A012340008B
S31508001A201B06C01880185A428018CA0F104349006E
S31508001A3007E04908C2071143DA05801A80194008E9
S31508001A40801800F003FBF8BD61000122511A001B43
S31508001A50F7E70122D2075140AAE70122D2075040F0
S31508001A60A6E7024670B54A40D30FDB0740002DD0E3
S31508001A704A002AD0010E140E000212020919400A61
S31508001A80520A8418E50104465443000A120A2E0431
S31508001A905043A4194219200CC543AA18120C012553
S31508001AA0AD03521C521912047F39240400D0521C6B
S31508001AB0104301D44000491EC2B20C06C0092018C2
S31508001AC0401C4008802A02D003E0002070BD400870
S31508001AD04000002900DA0020184370BD70B50246A0
S31508001AE04A40D50F40004A00ED0740085208002832
S31508001AF014D0002A12D0C40DD30D41020120C0050E
S31508001B005202490A520AE41A091812187D349142F7
S31508001B1001D3641C00E04900002C01DA002070BDE6
S31508001B200023914201D3891A03434008490000283B
S31508001B30F7D100290AD0914202D10121C90705E04F
S31508001B40914201D2012101E00121C943E005C018F3
S31508001B50401900F07BFA70BDF0B5074608465840B4
S31508001B6087B0C00F049048000E465900400849083F
S31508001B70BC1A884105D2384631461E4617460B46DA
S31508001B8002465800400810434CD0300D03904005DB
S31508001B905900400D490D0590401A0290402872DA06
S31508001BA018030121000B09050843019004980092C7
S31508001BB0002805D0019952420020884100920190E0
S31508001BC0029840210A1A0199009800F00BFA054676
S31508001BD00C466B4607CB00F026FAC0197141039AEA
S31508001BE00E0D0023D71756401A467A40164344D09E
S31508001BF0049A002A2DD0029A012A039A15DC1205A6
S31508001C00C01A914101263605001C7141D20F059E66
S31508001C10D2070093019202962A46234600F064FAF8
S31508001C2007B0F0BD38463146FAE71605224A0F4690
S31508001C30B218C01AB74101210905001C4F41001806
S31508001C407F41114618187941E20F10436D19644116
S31508001C5013E0E2076D0815436408C2071443039AA4
S31508001C6001261205C01A91413605001C7141CE079E
S31508001C70400830434908C01851412A46234600F017
S31508001C8026FACDE7FFE7049801224000C117121A89
S31508001C9000238B4104983146C417381AA141EEE750
S31508001CA030B40124E407634030BC55E730B401245E
S31508001CB0E407614030BC4FE70000E0FFF0B51FB411
S31508001CC088B00B990998002448400999C00F490023
S31508001CD049080991C0070B990090490049080B91DA
S31508001CE009990898A64608431CD00B990A980843F0
S31508001CF018D0099801244000420D4800410D099862
S31508001D0024050003000B204309900B980003000BE1
S31508001D1020430B9050181C49401800220190144685
S31508001D20104605E0002001460DB0F0BD032801DA93
S31508001D30034600E003239C46C11A0AAE0AE05F0088
S31508001D4008ADED5B4F00F75B7D430027AA187C4181
S31508001D50491C5B1E6145F2DD410004AB5A52210461
S31508001D60120C0A43240C401C0828DFDB0198029059
S31508001D700099704601910090059B049A0799069868
S31508001D8000F0B2F9D0E700000DFCFFFFF0B50C46F5
S31508001D905C4085B0E40FE40703944C000026640811
S31508001DA059009446490802460296224321D06246C3
S31508001DB00A431ED06200570D4A000E032303550D31
S31508001DC0012402462C492405781B1B0B360B4018A8
S31508001DD023432643614600901C46501AB44103D358
S31508001DE00098401C009002E0921800985B41002879
S31508001DF003DA0020014605B0F0BD002001210905DF
S31508001E000746864611E064461D46141BB54106D3AF
S31508001E106546521BB341744607430C43A646CD0795
S31508001E2040084908284392185B4105460D43EAD104
S31508001E301046184313D0604619465040714008436F
S31508001E4006D06046101AB34106D20122002306E0E6
S31508001E5000220123DB0702E00122D2435310009837
S31508001E6074460105381C6141029C039D00196941AD
S31508001E7000F02DF9BFE70000FD030000C217C10FEF
S31508001E80504010B54018CA079623002100F0E6F81E
S31508001E9010BD10B500229623114600F0DFF810BDDC
S31508001EA00EB5C217C10F5040CA0740180021054B8E
S31508001EB00293019200910A460B4600F015F903B009
S31508001EC000BD0000330400000EB50549029100214B
S31508001ED000910A460B46019100F006F903B000BDD1
S31508001EE033040000410040020122400AD205090ECF
S31508001EF080187F2901DA00207047962903DC96228C
S31508001F00511AC84070479639884070474A000903F5
S31508001F100123090B1B051943094B10B5520D9A42AB
S31508001F2001DA002010BD064B34339A4203DC9A1AB4
S31508001F3000F068F810BD03495118884010BD00002C
S31508001F40FF030000CDFBFFFFC20FD2074000400889
S31508001F500BD0C10D0723DB01C91840020905400A49
S31508001F601143C208400711437047002001467047D5
S31508001F7010B5002904DB0124E40740428C412146C0
S31508001F80002B04DB1C460123DB075242A3418B428C
S31508001F9000D1824210BD0000CB0FDB07490010B507
S31508001FA0490802460A4307D00A0D07240903E40133
S31508001FB0090B121B002A01DC002010BDC900440FC2
S31508001FC00C43C100E018D205801800F03FF810BD98
S31508001FD00122D207002800DB101A002900DB511A5B
S31508001FE08142704710B5202A04DB0146203A914009
S31508001FF0002010BD914020239C1A0346E340194354
S31508002000904010BD10B5202A04DB0846203AD0407F
S31508002010002110BD0B46D340D0402024A21A91407F
S315080020200843194610BD10B5202A06DBCB1708460B
S31508002030203A1041C1170B4306E00B461341D04026
S315080020402024A21A91400843194610BD002904DA33
S31508002050401C490001D140084000704770B4002474
S31508002060050C05D11024000402D1002921D0112421
S31508002070050E01D100020834050F01D10001241D07
S31508002080850F01D18000A41C002801DB4000641CD8
S31508002090002908D020252E1B0D46F540A14000D06A
S315080020A001212943084301061B1B000ADB1D02D533
S315080020B0002070BC7047DB05181880180029F8DA6C
S315080020C0401C4900F5D170BC40084000704710B567
S315080020D0002B08DA0024401C614192185B411A4320
S315080020E001D14008400010BDF0B51FB482B00546C6
S315080020F00C0003D0084602F045F902E002F042F966
S3150800210020300246009021462846FFF76BFF049BC5
S31508002110059A04460F4618431143084314D0184637
S3150800212010431BD0009840210A1A18460599FFF754
S3150800213069FF05460E46009A05990498FFF752FF6F
S31508002140084305D0012004E02046394607B0F0BD13
S315080021500020C11705430E432C43374300990E98B8
S315080021606305401A7905E40A00220C43FD0A0A3081
S3150800217002D500200146E9E70105101969410C9CC2
S315080021800D9D00196941FFF7A2FFDFE7FEB50023A1
S315080021901A461B1A8A4103DB0020014603B0F0BD2C
S315080021A04A000D0301212D0B0905520D0D43D107D8
S315080021B002D100186D41521E5110FF31FF31013115
S315080021C0002704463E4638460097019102460121FB
S315080021D000200905FFF716FFC3197141F8183246A2
S315080021E084468E464A4161462846611A904104D380
S315080021F06046241A954176461F46241900986D4173
S31508002200401C00903428E1DDF91930467041091B5D
S31508002210A84103D20022D243134601E00022134606
S3150800222001980105381C7141FFF751FFB6E7000018
S31508002230064C0125064E05E0E36807CC2B430C3C0B
S3150800224098471034B442F7D3FFF740FB6C66000892
S315080022508C66000810B50446002C08D10121092017
S31508002260C00600F0E3FD002000F0E6F852E0012C7D
S3150800227005D102210920C00600F0D8FD4AE0022C4B
S3150800228005D104210920C00600F0D0FD42E0032C48
S3150800229005D108210920C00600F0C8FD3AE0042C43
S315080022A005D110210920C00600F0C0FD32E0052C3A
S315080022B005D120210920C00600F0B8FD2AE0062C29
S315080022C005D140210920C00600F0B0FD22E0072C08
S315080022D005D180210920C00600F0A8FD1AE0082CC7
S315080022E004D101210D4800F0A1FD13E0092C04D109
S315080022F002210A4800F09AFD0CE00B2C04D11021AB
S31508002300064800F093FD05E00C2C03D18021034814
S3150800231000F08CFD204600F08FF810BD0004004840
S315080023207FB500200090019002900390002427E0DA
S3150800233000250CE0E800294940186100405AA10030
S315080023406A4651584018A1005050681C85B2142D91
S31508002350F0DBA1006A4650581421FFF7DBFA282162
S31508002360484361001E4A515A3C225143461864218B
S315080023703046FFF7CFFA6100194A5052601C84B202
S31508002380042CD5DB1748007A002826D01448408844
S315080023901549884203DC1248808888420ADD1148BC
S315080023A02038C07A002805D11049486001210D4817
S315080023B02038C1720A4840880A2803DB0848808802
S315080023C00A280ADA07482038C07A002805D10749BA
S315080023D04860012103482038C1727FBD48040020A7
S315080023E03C010020C0030020E60F0000C0010020C9
S315080023F000B587B001A800F0AFF80121480201F046
S3150800240051F800200190702002900120800203906C
S3150800241000200690059001A9064800F031F8012130
S31508002420044800F021F80121024800F011F807B02D
S3150800243000BD00000024014010B504460723002211
S315080024402146024800F038F810BD0000002401407B
S31508002450002904D0426801231A43426003E0426817
S315080024605208520042607047002904D08268082347
S315080024701A43826003E0826808239A4382607047A1
S3150800248042680B4B1A4042600B684A681A43436815
S315080024901A4342608268074B1A4082600B694A6990
S315080024A01A438B681A4383681A4382607047000090
S315080024B00FBCFFFF8FF1F9FFF0B504460D4616462F
S315080024C01F463F073F0F2B46082B0FD91B071B0F2D
S315080024D0083B606F9A000F21914088436067606FE0
S315080024E099003A468A40104360670BE0206F9A00CD
S315080024F00F21914088432067206F99003A468A4009
S3150800250010432067E0680121A9408843E060E0683D
S315080025100121A9400843E0600120800328400028E3
S3150800252003D0012000F020F807E00120C00328406E
S31508002530002802D0012000F017F8F0BD002905D0C8
S315080025408268FF2301331A43826004E08268FF230E
S3150800255001339A43826070470021016041608160BF
S315080025600173016141617047002806D00649496830
S315080025700C221143044A516005E0034949680C22BC
S315080025809143014A516070470024014010B5244820
S315080025900078012834D10020214908702149088093
S315080025A012E02048008840001F49085A1F49098838
S315080025B0C9001F4A89181B4A1288520088521948AE
S315080025C00088401C17490880164800880428E8DB5C
S315080025D07E2001F087FE022000F02EF90121154821
S315080025E0FFF7ACFF11480088401C104908800846D0
S315080025F00088142804DB0020088001200E49087092
S315080026000D480078002806D0FFF78AFE00200A4900
S31508002610087000F055FC7E2001F064FE10BD000035
S315080026204C010020660100201004002068010020EB
S31508002630480400200024014044010020FFB583B06F
S315080026400C46029400200190002726E000261CE094
S31508002650721C039951430846791CFFF75BF9054636
S31508002660A54201D9281B00E0601B05460298A8422E
S3150800267004D90295059806700698077002980028EE
S3150800268002D10120019002E0761C402EE0D300BF63
S315080026900198002800D002E07F1C042FD6D300BF83
S315080026A0029807B0F0BD000000BF00BF00BF00BF22
S315080026B000BFBFF34F8F00BF00BF00BF06480749E2
S315080026C0C86000BF00BF00BFBFF34F8F00BF00BF89
S315080026D000BF00BF00BFFDE70400FA0500ED00E0FB
S315080026E010B500F001F810BD10B523480078002891
S315080026F017D1224800F05EFF01283CD11F48007818
S31508002700002838DD1D480078402834DC01F0C1FA7D
S315080027101B490860012018490870002019490870EB
S3150800272029E0164A17490978491C501800F042FF53
S31508002730012816D113480078401C124908700F4822
S3150800274000780978884216D100200B4908700B4892
S315080027504078FF280FD10B48007802280BD1FFF7E5
S31508002760A3FF01F096FA064909686431884202D93E
S3150800277000200149087010BD15010020CC03002077
S31508002780180100201401002010B586B00446012166
S31508002790880300F087FE0121480400F063FE012249
S315080027A00921C80600F02DFB01220A210920C006CE
S315080027B000F027FB01A801F072FB0194302168465E
S315080027C0018100214181818101821821C18101A9EC
S315080027D0184801F021FB0121164801F0FAFA05A86C
S315080027E000F065FB01214902684681820121817555
S315080027F01821C17505A90920C00600F0B5FA0121FE
S315080028008902684681824821C17505A90920C00642
S3150800281000F0AAFA1B2168460170032141700121C4
S31508002820817000F0EBFD01220221024801F0E9FA6D
S3150800283006B010BD0038014001B50449009808608B
S3150800284000BF024800680028FBD108BD1C01002013
S31508002850014600220E4B1A61CA005A6100229A618B
S3150800286005221A6100BF0A4A1069C207D20F002A58
S3150800287004D0012212040240002AF4D0044A126944
S3150800288052085200024B1A6100229A6170470000F2
S3150800289000E000E010B500210448FFF74FFE0220D3
S315080028A000F04AF801200249087010BD00240140D2
S315080028B04C01002000B589B00121084600F0D2FD80
S315080028C01A4800F045F801A800F08EF8184801905B
S315080028D0184802900021684601730420049068464F
S315080028E00175802141754900C18289000183202133
S315080028F08176090281830021C183018401A90B48DD
S3150800290000F04CF80121094800F01CF801220221C8
S31508002910064800F039F8092168460170022141701D
S315080029200121817000F06AFD09B000BD080002406F
S315080029300024014010040020014948607047000047
S31508002940000002400268520852000A4302607047BB
S3150800295010B504462068400840002060002020602A
S315080029606060A060E060E1B2084608380521FEF71D
S31508002970D1FF01460F2088400249496808430149AA
S31508002980486010BD00000240002A03D003680B43CC
S31508002990036002E003688B430360704710B50A7A48
S315080029A08B7D1A430B7C1A434B7C1A434B8A1A437A
S315080029B08B8A1A430B8B1A434B8B1A430368094CB1
S315080029C023401A43026002680123DB039A438B8B78
S315080029D01A430260CA6842600A6882604A68C2602E
S315080029E010BD00000F80FFFF0021016041600172E9
S315080029F0C16001744174418281828175018341837A
S31508002A008183704770B506460C4621460A4800F091
S31508002A104BF90546002D01D1401E70BD064885427A
S31508002A2002D10648051B00E02D1B224629463046E2
S31508002A30FEF79AFF2046F0E700F4000800FC0008BD
S31508002A4070B506460C4621460A4800F02DF905469B
S31508002A50002D01D1401E70BD0648854202D10648A8
S31508002A60051B00E02D1B224629463046FEF77CFF53
S31508002A702046F0E7008000080088000870B5064682
S31508002A800C4621460A4800F00FF90546002D01D1EB
S31508002A90401E70BD0648854202D10648051B00E067
S31508002AA02D1B224629463046FEF75EFF2046F0E7F4
S31508002AB0009000080098000870B505460C462246A6
S31508002AC00249284600F0B1F8204670BD00F4000817
S31508002AD070B505460C4622460249284600F0A5F878
S31508002AE0204670BD0080000810B5044608480069F5
S31508002AF002210843064908610846446100694021E5
S31508002B00084303490861034800F00EF910BD0000A8
S31508002B1000200240FF0F00000C48C068C007C00F25
S31508002B20002801D0012070470848C06804210840E1
S31508002B30002801D00220F6E70448C06810210840A2
S31508002B40002801D00320EEE70420ECE7002002402D
S31508002B50034800698021084301490861704700005D
S31508002B600020024030B504460D460548006901219B
S31508002B7008430349086125800F2000F0D5F830BDC9
S31508002B800020024010B57E2001F0ACFB064800F09C
S31508002B900FF87E2001F0A6FB044800F009F87E2015
S31508002BA001F0A0FB10BD000000F40008008000083A
S31508002BB010B5044600F0ACF82046FFF795FFFFF77E
S31508002BC0C7FF10BD70B503460125002208E0500076
S31508002BD01C5A0748844201D0002506E0501C82B2E0
S31508002BE0CE0F761876109642F1DC00BF284670BDE7
S31508002BF0FFFF0000F8B505460E46144600F088F8B3
S31508002C007E2001F06FFB002707E029883046FFF792
S31508002C10A9FFB61CAD1C781C87B2E10F091949102B
S31508002C20B942F2DCFFF794FFF8BDF8B507460C4643
S31508002C3015462946204600F037F80646002E0DD1DF
S31508002C402046FFF7B5FF012080022018FFF7B0FFE6
S31508002C502A4621463846FFF7CDFF24E001208002A8
S31508002C602018401BB0420AD1012080022018FFF725
S31508002C709FFF2A4631463846FFF7BCFF13E001207E
S31508002C80C0022018401BB04208D12046FFF790FF2B
S31508002C902A4631463846FFF7ADFF04E02A46314654
S31508002CA03846FFF7A7FFF8BDF8B505460E462F4686
S31508002CB0E807C00F002801D000BFFEE73146012013
S31508002CC0C002FEF73DFE002901D000BFFEE7002442
S31508002CD00BE020467043471931463846FFF772FF26
S31508002CE0012800D108E0601C84B231460120C002E8
S31508002CF0FEF726FEA042ECDC00BF31460120C002EA
S31508002D00FEF71EFEA04200D100273846F8BD000097
S31508002D1002480349486003484860704723016745ED
S31508002D2000200240AB89EFCD10B5024600BFFFF781
S31508002D30F3FE0346521EFF2400E0641E002CFCD15D
S31508002D40012B01D1002AF2D1064800697721884370
S31508002D50044908613420C860002A01D1052010BD45
S31508002D601846FCE700200240F8B50246CD782F0742
S31508002D703F0FCD7810263540002D01D08D782F4392
S31508002D801446002011E085062B0E0D880126864084
S31508002D903540002D07D025680F269E40B5433E4690
S31508002DA09E4035432560451CE8B20828EBDB141D18
S31508002DB00D882D120095002011E085062B0E0125A1
S31508002DC08540009E3540002D07D025680F269E4079
S31508002DD0B5433E469E4035432560451CE8B2082863
S31508002DE0EBDBCD78282D04D155690E88354355611E
S31508002DF006E0CD78482D03D115690E88354315614F
S31508002E00F8BD70B54D07EB0E082902DA05462035E0
S31508002E1001E0054624352C460F269E402568B54315
S31508002E2016469E403543256070BD000038B50446F9
S31508002E300D460920C006844203D10121480400F04A
S31508002E4011FB1148844203D10121000200F00AFB5C
S31508002E500E48844203D10121000200F003FB0C480E
S31508002E60844203D10121080500F0FCFA684600F007
S31508002E701EF868460580012181700021C1706946E7
S31508002E802046FFF771FF38BD0004004800080048D7
S31508002E90000C0048024690680840002801D001202E
S31508002EA070470020FCE741617047016170470021C7
S31508002EB0C9430180022181700421C1707047000056
S31508002EC0F0B58FB00025002600200D900C907E20CE
S31508002ED001F008FA00241AE06100A94A505AFEF7E0
S31508002EE0D8FFA8490790FEF7F9FD0746FFF72CF823
S31508002EF00022A54B09910890FEF7E0FE0B910A9077
S31508002F00FFF74AF8A100A14A5050601C84B2042C6D
S31508002F10E2DB9E498868FFF717F89D4A9D4B0591A5
S31508002F200490FEF7BDFE00229B4B07910690FEF724
S31508002F302DFF9A4A9A4B09910890FEF7B7FE0B9116
S31508002F400A90FFF729F8054690494868FEF7FCFFFE
S31508002F508F4A904B05910490FEF7A2FE00228E4BF5
S31508002F6007910690FEF712FF8C4A8D4B099108903F
S31508002F70FEF79CFE0B910A90FFF70EF806462846C8
S31508002F80FEF7E2FF0022874B05910490FEF78EFEBE
S31508002F900991089029468448FEF763FD0746FEF71F
S31508002FA0D3FF07910690099B089AFEF7EFFE0B914F
S31508002FB00A90FEF7F1FF7D4908603046FEF7C4FF28
S31508002FC00022784B05910490FEF770FE099108904F
S31508002FD031467548FEF745FD0746FEF7B5FF0791EA
S31508002FE00690099B089AFEF7D1FE0B910A90FEF708
S31508002FF0D3FF6F4908606F49088BFEF765FF6E4A75
S315080030006E4B03910290FEF759FE00226C4B059118
S315080030100490FEF7BBFE099108906649088BFEF7F7
S3150800302038FF0746FEF790FF0022654B0191009096
S31508003030FEF7ACFE059104905C480068FEF784FF35
S3150800304003910290059B049AFEF72AFE07910690C3
S31508003050099B089AFEF79AFE0B910A90FEF79CFFC9
S315080030600D905449488BFEF72FFF534A534B039153
S315080030700290FEF723FE0022514B05910490FEF7BD
S3150800308085FE099108904B49488BFEF702FF0746D3
S31508003090FEF75AFF00224A4B01910090FEF776FE92
S315080030A00591049042480068FEF74EFF039102908E
S315080030B0059B049AFEF7F4FD07910690099B089A6A
S315080030C0FEF764FE0B910A90FEF766FF0C903D48EA
S315080030D00D99FEF76DFC0746FEF704FF3A490860AE
S315080030E038480C99FEF764FC0746FEF7FBFE37499D
S315080030F008603748808A344909684018C003010CBB
S3150800310033488182C08A314909684018C003010CD6
S315080031102F48C1821D49C8682E49FEF7A2FC0746FA
S31508003120FEF7E0FE81B22A488184FF38C13800885C
S31508003130FF21F531884220DD00201E4954390880D8
S31508003140124908682449FEF743FF11D22048203067
S31508003150C07A002806D117495439486001211C480D
S315080031602030C172FF2101311C48FFF79EFE04E0A2
S31508003170FF2101311948FFF796FE0FB0F0BD000098
S315080031803C01002000F07F4500000840380400207C
S31508003190333333333333C33F000028404A0C022B02
S315080031A08716D13F00000440000048435401002020
S315080031B05801002014020020091B9E5E29CB703F8F
S315080031C000408F400000C8415C01002060010020DB
S315080031D0800300200000C8427B142E3F00040048EC
S315080031E00148006870470000200100200348006875
S315080031F003490978401801490860704720010020F2
S315080032002801002008B50121480400F02BF9012106
S31508003210880400F027F96846FFF749FE0121C9032B
S31508003220684601804821C17069460920C006FFF733
S315080032309BFD6846FFF73BFE0121090368460180AE
S315080032404821C17069460920C006FFF78DFD68460A
S31508003250FFF72DFE4021684601800421C1706946AA
S315080032600148FFF781FD08BD0004004810B501219B
S31508003270C9030920C006FFF70DFE002839D13E48CC
S31508003280807B002839D13C48407A01282CD13A481D
S315080032902030007A002827D137482030C079401CD2
S315080032A0C1B235482030C171C07904281CDB202101
S315080032B03248FFF7FAFD00212F482030C171AC389B
S315080032C04089002807D12E482E49486001212A48FE
S315080032D08C38418106E000202A49486000212648AA
S315080032E08C38418101F01EF80121234881738172CF
S315080032F003E00021204881728173224880682049B2
S31508003300884232D900201F49886000211A488172F4
S315080033102030007A002822D108211848FFF7C5FD79
S3150800332015488C384088032811DA13488C384089A8
S3150800333000280CD110482038C08A822804DA0121D6
S315080033400D482030017202E001210B48C1720A487B
S31508003350407A012809D100200A49486005E0002082
S31508003360084948600021044841727E2000F0BAFFEF
S315080033700148807A10BD0000A00300200004004820
S31508003380DC050000C001002008B50121480400F052
S3150800339069F80121880400F065F86846FFF787FD9B
S315080033A0FF212A3168460180012181701021C170F0
S315080033B069461148FFF7D8FCB62168460180012105
S315080033C081701021C17069460920C006FFF7CCFC40
S315080033D010210920C006FFF766FD80210920C006D6
S315080033E0FFF761FD01210448FFF75DFD082102484A
S315080033F0FFF75BFD08BD000000040048817800293E
S3150800340025D01749032212028918027892109200D1
S31508003410895802789207D30EFF229A409143427840
S315080034209207120E03789B07DB0E9A4011430C4A4B
S3150800343003231B02D21803789B109B00D1500178F6
S31508003440CA06D20E01219140054A116007E00178AB
S31508003450CA06D20E01219140014A80321160704796
S3150800346000E100E0002905D0054A52690243044BF1
S315080034705A6104E0024A52698243014B5A61704715
S3150800348000100240002905D0054AD2690243044BC0
S31508003490DA6104E0024AD2698243014BDA61704775
S315080034A000100240002905D0054A92690243044BE0
S315080034B09A6104E0024A92698243014B9A61704715
S315080034C00010024010B500F031F804494968F022AE
S315080034D011400909024A515CC84010BD001002405B
S315080034E0EE00002010B5FFF7EDFF054949680722F1
S315080034F012021140090A034A515CC84010BD000077
S3150800350000100240EE00002010B5FFF7DBFF05496A
S3150800351049680722D2021140C90A034A515CC840C9
S3150800352010BD000000100240EE000020F8B51E484D
S3150800353040680C210840042802D008282ED101E052
S315080035401A4C2DE0184840300069C007C00F002803
S315080035500AD015484030006902210840002801D0E9
S31508003560134802E0114800E0104807460E4840306C
S315080035700069FF2109040840000C451C0A48403030
S315080035800069072109020840000A461C39466943B2
S3150800359008463146FEF7BEF9044601E0034C00BF73
S315080035A000BF2046F8BD00000010024000127A0055
S315080035B000093D0070B5044600250221074800F0C1
S315080035C00EFC002808D0054800F062FC2070022195
S315080035D0024800F0FCFB0125284670BD0038014072
S315080035E010B500F001F810BD00B585B06248006856
S315080035F0012108436049086000BF5F48006802214E
S3150800360008400028F9D05D485D4908605D480068B3
S31508003610102108435B49086008460068C008C000D6
S31508003620086057490968481E5749FEF773F9049018
S315080036305448006804994907490F084351490860E6
S315080036404D484068514908404B494860084640681B
S3150800365090210843484948600846406848604848F9
S3150800366000684649884207D9434840680521090247
S315080036700843414948600BE041480068444988428C
S3150800368006D93D4840680121890208433A494860FD
S315080036906B4601AA3A4801683E48FEF7CFFF36480E
S315080036A04030006980088000334940310861084687
S315080036B00069400840000861684600784007400FE6
S315080036C00290684600794006400E03902A48C06971
S315080036D0890508432849C8612748403000692E49AA
S315080036E008402549403108610398000402990902F7
S315080036F0084321494031096908431F494031086197
S315080037001D4800680121090608431B49086000E0B6
S3150800371000BF194800680121490608400028F7D06B
S315080037201548406880088000134948600846406884
S31508003730022108431049486000E000BF0E4840686F
S315080037400C2108400828F8D10120FFF781F80A481B
S31508003750406810218843084948600120FFF778F837
S315080037600548406880218843034948600120FFF7DF
S315080037706FF805B000BD00000010024000A24A0420
S31508003780000100200020024000366E010FC0FFFF36
S315080037900051250200127A00FFF800FF042806D11E
S315080037A00649096904221143044A116105E00349DF
S315080037B0096904229143014A1161704700E000E05B
S315080037C010B5FFF713FD59480088401C5749088073
S315080037D008464068401C486055480068002804D0E0
S315080037E053480068401E524908605248807A0128AA
S315080037F005D14E488068401C4C49886002E000208C
S315080038004A4988604B48C079012805D1474800696C
S31508003810401C4649086102E00020444908614548C1
S31508003820007B012805D14148C06B401C3F49C8634D
S3150800383002E000203D49C8633C4948680A21FEF772
S3150800384069F8002923D13B482030C1788078814225
S3150800385008DD384820308078401CC1B23548203011
S31508003860817014E033482030C1788078814200D1D5
S315080038700DE030482030C1788078814207DA2D483B
S3150800388020308078401EC1B22A48203081702948ED
S315080038902030007A022804D026482030007A0328EF
S315080038A004D12248406B401C2049486321482030F7
S315080038B0407900280AD11F482030007A042805D10B
S315080038C01A48406C401C1949486402E00020174910
S315080038D048641848C07B012805D11448C06C401CB0
S315080038E01249C86402E000201049C8641148007CE7
S315080038F0012805D10D48806C401C0C49886402E0FB
S3150800390000200A4988640B48807904280AD10748A8
S31508003910006D0949884208D20448006D401C0349D5
S31508003920086502E000200149086510BDC0010020B5
S315080039301C010020A003002050C3000010B5164843
S31508003940006801210843144908600846406813497D
S3150800395008401149486008460068114908400E4960
S315080039600860084600680121890488430A490860F6
S3150800397008464068C3210904884307494860084641
S31508003980006808490840044908609F2000048860C8
S31508003990FFF726FE10BD0000001002400CC0FFF81D
S315080039A0FFFFF6FEFFFF8F0008B501214804FFF769
S315080039B059FD022201210920C006FFF722FA022139
S315080039C0684601801821C170012181706946092065
S315080039D0C006FFF7C9F901214804FFF743FD022293
S315080039E011460920C006FFF70CFA04216846018033
S315080039F01821C1700121817069460920C006FFF7A8
S31508003A00B3F908BD30B587B004460D46012108460E
S31508003A10FFF738FD04A800F033F9059468460582D7
S31508003A20002101838176817404A90120800700F0B2
S31508003A30F1F8684600F0D2F8602168460170012165
S31508003A4041700020019000216846017269460120F4
S31508003A50800700F057F869460120800700F08AF8C9
S31508003A600821C80600F07EF80821C80600F0B0F85C
S31508003A704021080600F038F84021080600F03CF816
S31508003A800121880700F00AF80121880700F01EF8CE
S31508003A900121880700F00EF807B030BD002904D0D0
S31508003AA0026880231A43026003E0026880239A436F
S31508003AB002607047002904D0026801231A43026095
S31508003AC003E002685208520002607047002905D0D8
S31508003AD0426C0123DB031A43426404E0426C01236F
S31508003AE0DB039A4342647047826907231B039A43A0
S31508003AF00B021A4382617047C26970239A430A43CC
S31508003B00C261704710B5826907231B039A430B7875
S31508003B101B021A4382610A7A12014B781B011A4367
S31508003B20036A3024A3431A4302624A6882630C4A32
S31508003B30904213D14A7A12018B781B011A43036A01
S31508003B40C024A3431A4302624A8992008B899B00C8
S31508003B501A4343682401A3431A43426010BD000078
S31508003B60002C014082690123DB029A430B021A43A7
S31508003B708261704710B5C26970239A430B781A435D
S31508003B80C2610A7A12024B781B021A43036A03249B
S31508003B902402A3431A4302624A68C2630B4A90424C
S31508003BA013D14A7A12028B781B021A43036AA400BD
S31508003BB0A3431A4302624A8912018B891B011A43DD
S31508003BC04368A400A3431A43426010BD002C014079
S31508003BD0C26908239A430A43C261704700210170EB
S31508003BE041708170416001724172418181817047E3
S31508003BF001229207904201D1816301E08AB2826371
S31508003C00704701229207904201D1C16301E08AB24E
S31508003C10C2637047026803231B029A430B891A433F
S31508003C200260134A904206D001229207904202D0BF
S31508003C30104A904205D1026870239A438B781A433A
S31508003C4002600B4A904205D00B4A904202D00B4ABA
S31508003C50904205D1026B120A12028B7A1A4302634A
S31508003C604A68C2620A88826201224261704700007D
S31508003C70002C014000040040004401400048014077
S31508003C800021C94341600021018001818170817250
S31508003C90704710B5FFF7A4FA10BD000070B5FFF71E
S31508003CA011FC05467D21C900FDF734FE0446601E59
S31508003CB00C49884200D90CE0601E0B494861032173
S31508003CC0081F00F085FB0020074988610720086166
S31508003CD000BF0420FFF762FD0021481E00F078FBB4
S31508003CE070BD0000FFFFFF0000E000E010B50221F4
S31508003CF0154800F07DF8002824D0134800F0C8F8CD
S31508003D00C4B21248C079002803D1204600F06EFFDD
S31508003D1014E00E48C079022810D10C48007A002811
S31508003D200CD10B488079AA2804D10948C47101210D
S31508003D3006480172AA2C01D105488471022102485D
S31508003D4000F045F810BD000000380140A00300202F
S31508003D50F804002010B504462146054800F09CF8F2
S31508003D6000BF0121024800F03AF80028F9D010BD3A
S31508003D700038014070B505460E4600247E2000F046
S31508003D80B1FA00BF20E0042C19DD701EA04216DD32
S31508003D90285D7E2806D17D20FFF7DCFF5E20FFF731
S31508003DA0D9FF0FE0285D7D2805D1FFF7D3FF5D20F9
S31508003DB0FFF7D0FF06E0285DFFF7CCFF02E0285D9D
S31508003DC0FFF7C8FF601C84B2B442DCDB70BD4161FA
S31508003DD070478269520852000A4382617047024658
S31508003DE090680840002801D0012070470020FCE7B1
S31508003DF00246D0680840002801D0012070470020FC
S31508003E00FCE7002A03D003690B43036102E0036958
S31508003E108B4303617047000070B504460D460026C3
S31508003E20E0693021884329790843E061E069442143
S31508003E308843A9790843E061E06980088000297A07
S31508003E400843E061A0691821884369890843A0618D
S31508003E50A06904218843297B0843A0610B48844252
S31508003E6003D1FFF751FB064602E0FFF73BFB064688
S31508003E7030462968FDF74EFD00092062304629685C
S31508003E80FDF748FD0007000F606270BD003801406D
S31508003E9001464868C0B27047CAB2026070474B21F3
S31508003EA0C901016030210171002181710172182157
S31508003EB0418100210173704710B51C4840880300F2
S31508003EC000F077FA0504111E292A2B0017486C30D2
S31508003ED0808CFF211B31884204DA01211348418076
S31508003EE000F020FA19E011486C30808CFF2105316A
S31508003EF0884204DA02210D48418000F013FA0CE0EA
S31508003F000A486C30808CFD2804DA03210748418072
S31508003F1000F008FA01E000E000BF00BF03488C305B
S31508003F20407A002801D100F0FDF910BD14030020E5
S31508003F3010B530484088002806D0012813D002283A
S31508003F4020D0032854D12CE080210920C006FEF792
S31508003F50ACFF01212848FEF7A8FF10210920C0065A
S31508003F60FEF7A3FF44E001212348FEF79EFF8021C8
S31508003F700920C006FEF797FF10210920C006FEF7A4
S31508003F8092FF35E080210920C006FEF78EFF012149
S31508003F901948FEF788FF10210920C006FEF783FF9F
S31508003FA026E016494868CD21FDF7B4FCC007C00FC6
S31508003FB0002805D080210920C006FEF774FF0DE011
S31508003FC00E494868CD21FDF7A5FCC007C00F00289B
S31508003FD004D180210920C006FEF767FF01210648A3
S31508003FE0FEF761FF10210920C006FEF75CFF00BF3F
S31508003FF000BF10BD1403002000040048C0010020C3
S3150800400010B5A0488079030000F0D3F90504336C95
S31508004010AFFDFC009B482038808CFF210531884283
S3150800402002DB01219748817140219748FEF732FF4C
S3150800403000281DD095494868FF21F531FDF76AFC2F
S31508004040C007C00F002805D180210920C006FEF749
S315080040502AFF04E080210920C006FEF726FF10216A
S315080040600920C006FEF71FFF01218748FEF71BFF40
S3150800407006E184482038808CFF211B31884202DB08
S3150800408002218048817140217F48FEF703FF0028FE
S3150800409027D07E494868FF21F531FDF73BFCC0076C
S315080040A0C00F002804D101217748FEF7FCFE03E083
S315080040B001217548FEF7F9FE80210920C006FEF7A2
S315080040C0F2FE10210920C006FEF7EDFE6D488C3879
S315080040D04088012805D001216A488C38418000F0C3
S315080040E021F9CDE067482038808CFF2125318842A8
S315080040F002DD03216348817140216348FEF7CAFE49
S31508004100002831D061494868FF21F531FDF702FCE6
S31508004110C007C00F00280ED180210920C006FEF76F
S31508004120C4FE01215848FEF7C0FE10210920C0062A
S31508004130FEF7BBFE0DE080210920C006FEF7B3FEA0
S3150800414010210920C006FEF7AEFE01214E48FEF7F3
S31508004150AAFE4C488C384088002805D000214948DA
S315080041608C38418000F0DEF88AE040214648FEF7A8
S3150800417091FE00284ED0012109030920C006FEF74A
S3150800418089FE002811D080210920C006FEF78DFE81
S3150800419001213D48FEF789FE10210920C006FEF7D9
S315080041A084FE04213748817126E038494868FF2192
S315080041B0F531FDF7AFFBC007C00F00280ED18021EF
S315080041C00920C006FEF771FE01212F48FEF76DFE95
S315080041D010210920C006FEF768FE0DE0802109209F
S315080041E0C006FEF760FE10210920C006FEF75BFE3A
S315080041F001212548FEF757FE22488C3840880028BA
S3150800420008D001E03BE006E000211E488C384180DA
S3150800421000F088F834E040211B48FEF73BFE0028F2
S315080042202CD018488C384088002805D0002115481D
S315080042308C38418000F076F81448006D144988429D
S315080042400ED280210920C006FEF72FFE01210E4856
S31508004250FEF72BFE10210920C006FEF726FE0DE00C
S3150800426080210920C006FEF71EFE10210920C0067F
S31508004270FEF719FE01210448FEF715FE00E000BF0F
S3150800428000BF10BDA003002000040048C0010020A4
S31508004290307500000348806840084000014988607E
S315080042A070470000002C004080210143014A11603C
S315080042B070470000002C004003488068002801D0A1
S315080042C0012070470020FCE7002C004010B5FFF7DE
S315080042D0F3FF002804D0FFF7DDFF662000F002F8A0
S315080042E010BD00004106490E014A116070470000E2
S315080042F0002C004004494968FF228132914301435A
S31508004300014A516070470000002C00400449496882
S31508004310C909C9014206520E1143014A5160704744
S31508004320002C004010B57E20FFF7DCFF0948FEF799
S315080043303FFC0949094881820621143000F09AF8A1
S315080043400649143188814022024904481430FEF790
S315080043506CFC10BD00900008FBAA000000030020BA
S3150800436070B505460C460121C802FFF78BF8FF20F9
S315080043708130FFF7BFFF2046FFF7C8FF2846FFF743
S3150800438093FF70BD2021020C01D010211046020AAD
S3150800439001D010460839020901D01046091F8208C3
S315080043A001D01046891E420801D0881E7047081A97
S315080043B0704730B47446641E2578641CAB4204D337
S315080043C0635D5B00E31830BC18471D46F8E700003C
S315080043D010B5002819DB1A4A03231B02D2188308D2
S315080043E09B00D2588307DC0EFF23A3409A438B0712
S315080043F01B0E8407E40EA3401A43114B0324240220
S315080044001B198408A4001A5118E00E4A03071B0F4B
S31508004410083B9B089B00D2588307DC0EFF23A3406A
S315080044209A438B071B0E8407E40EA3401A43054BD9
S315080044300407240F083CA408A4001A5110BD000064
S3150800444000E100E01CED00E002E008C8121F08C108
S31508004450002AFAD170477047002001E001C1121FF7
S31508004460002AFBD170470000014908607047000028
S31508004470BC01002010B502460023002901D1002006
S3150800448010BD03E01488921CE01883B208464C1E3F
S31508004490A1B20028F6D11846F2E70000F8B50027C1
S315080044A0002600240025FC48007A01286FD17E20CA
S315080044B0FFF718FFF948C0790002F849097A084356
S315080044C00746F648467A847A0246D17A107B00F087
S315080044D0CBFC05460021F0480172F149781A8F4253
S315080044E06FD01EDCEF49781A8F426BD010DCEE498C
S315080044F0781A8F4267D006DC442F1CD0EB48381850
S31508004500002872D1E4E1882870D08928F9D174E1AD
S3150800451001286CD002286BD003286AD00428F0D171
S3150800452035E10300FFF745FF0C61C0FAF861611930
S3150800453026768E415C61062E09D1DD480078002872
S315080045400AD100F037FF0120D949087004E0152E7A
S3150800455002D1012000F02EFFD5E1CF482030007AA5
S31508004560002806D0CC482038828AC18A002000F06C
S315080045707BFEC8E1002C0BD1C7482038C08A00232F
S315080045801A46F0210090FE2000F0A3FE0CE0BBE1E5
S31508004590012C09D1C0482038808A01230022F02145
S315080045A00090FE2000F095FEADE1002C0CD1C1482C
S315080045B0408800231A46F3210090FE2000F089FE69
S315080045C00DE05AE05BE18EE1012C08D1B9488089FB
S315080045D001230022F3210090FE2000F07AFE92E1EA
S315080045E0002C07D1B348458006E08BE119E122E1AA
S315080045F06AE07AE0AF488581AE488089FF21F531C7
S31508004600884206DA00F0D0FA0022FE21F42000F0F3
S3150800461094FE78E1002C09D1A648808800231A4622
S31508004620F1210090FE2000F054FE0AE0012C08D18A
S31508004630A048C08901230022F1210090FE2000F045
S3150800464048FE60E1002C02D19A48858003E0012CDF
S3150800465001D19848C58197488088FF21F53188425D
S315080046600ADC9448C089884206DC00F09DFA0022DC
S31508004670FE21F22000F061FE45E1002C09D18D48AB
S31508004680C08800231A46E9210090FE2000F021FE8A
S3150800469009E0012C07D1192001230022E921009005
S315080046A0FE2000F016FE2EE1002C01D18148C580BF
S315080046B0FF202D30854206DA00F076FA0022FE2128
S315080046C0EA2000F03AFE1EE1002C0CD17948008958
S315080046D06421484380B200231A46E2210090FE2056
S315080046E000F0F7FD00E000BF0DE1002C06D16421C3
S315080046F02846FDF725F981B26E4801816D48008983
S31508004700FF21F531884206DC00F04EFA0022FE2130
S31508004710E32000F012FEF6E01EE0FFE7002C0CD1C5
S31508004720644840896421484380B200231A46EB2135
S315080047300090FE2000F0CDFD0DE0012C0BD15D4868
S31508004740008A6421484380B201230022EB210090AD
S31508004750FE2000F0BEFDD6E0002C07D164212846D5
S31508004760FDF7EEF881B25348418108E0012C06D1E5
S3150800477064212846FDF7E4F881B24E48018200F02C
S3150800478013FA0022FE21EC2000F0D7FDBBE0012C35
S315080047901AD141488C38408803280CDA3E488C38B0
S315080047A04089002807D101213B48203001720020AA
S315080047B04049543948600022FE21E42000F0BDFD3E
S315080047C001213548417217E0002C10D100213248EA
S315080047D04172203001720022FE21E42000F0ADFD76
S315080047E000203349087033495439486004E00022F0
S315080047F0FE21E42000F0A1FD85E0002C0FD127481A
S31508004800C07A32280CDC2548C17A2A48418200F051
S31508004810CBF90022FE21DF2000F08FFD00E000BF6B
S3150800482071E02448408A00231A46DE210090FE20C3
S3150800483000F04FFD67E0002C0FD11848C07A3228E7
S315080048401CDC1648C17A1B48818200F0ADF90022AB
S31508004850FE21E12000F071FD10E0012C0ED10F4879
S31508004860C07A32280ADC0D48C17A1248C18200F0A3
S315080048709BF90022FE21E12000F05FFD43E0002CB9
S315080048801AD10C48808A00231A46E0210090FE209F
S3150800489000F01FFD1BE00000A0030020F804002024
S315080048A0E9FE0000E0FE000056FE0000AB01FFFF37
S315080048B0B801002014020020012C08D11348C08A30
S315080048C001230022E0210090FE2000F002FD1AE0FC
S315080048D0002C07D101210E48C171002202210D4882
S315080048E0FFF78FFA0FE0002C0BD1FF2101310A48A0
S315080048F0FDF753F800200849891F0880022104485B
S31508004900C17100E000BF00BFF8BD0000140200201E
S31508004910A003002000380140FE040020F0B589B04D
S3150800492000200890079006903848007A01286BD135
S3150800493037488079AA2864D13548C079322860DAA0
S315080049403348C07900285CDD3149C97908461938E9
S31508004950FDF794FA08900898FDF7F6FA04462D4AEA
S315080049602D4BFDF7ABF900222C4B01910090FDF77A
S31508004970F3F8039102902A480068FDF7E5FA06461F
S31508004980039B029AFDF702FA05910490FDF704FBD2
S31508004990079024490798FDF764F80446FDF7A2FA3C
S315080049A081B2214801830898FDF7CEFA0646194ACE
S315080049B0194BFDF783F904460022184BFDF7CCF88E
S315080049C00391029019480068FDF7BEFA019100901C
S315080049D0039B029AFDF7DAF905910490FDF7DCFAD4
S315080049E0069010490698FDF73CF80446FDF77AFA52
S315080049F081B20D48418300F0D7F800210348C17100
S31508004A00417200210148017209B0F0BDA0030020DF
S31508004A10F8040020091B9E5E29CB703F0000F03F7A
S31508004A205401002000007A44140200205801002096
S31508004A3070B505460E461446002E02D0012E4AD100
S31508004A4020E0002D02D0012D1AD10CE060210120B2
S31508004A508007FFF749F8002101208007FFF7C8F80B
S31508004A601E4804700CE0602101208007FFF744F817
S31508004A70002101208007FFF7C4F81948047000BF19
S31508004A8000BF28E0002D02D0012D22D110E01348E6
S31508004A900078A0420BD0602101208007FFF724F898
S31508004AA0214601208007FFF7A3F80C48047010E0A0
S31508004AB00B480078A0420BD0602101208007FFF741
S31508004AC01BF8214601208007FFF79BF8044804706D
S31508004AD000BF00BF00BF00BF70BD00006A01002014
S31508004AE06B01002010B5052421E080212C48FCF735
S31508004AF054FF80212A48FDF785FF0F212848FFF734
S31508004B00B9FC2749C98B88420CD125481438808AB4
S31508004B102449884204D000F0CFF900F045F800E0B7
S31508004B2010BD04E0002000E0401C8028FCDB204685
S31508004B30611ECCB20028D8D100BF052423E080210D
S31508004B401748FCF72AFF80211548FDF779FF0F2142
S31508004B501348FFF78FFC1249C98B88420ED11048BB
S31508004B601438808A0F49884204D000F0A5F900F06D
S31508004B701BF802E000F018F8D2E704E0002000E095
S31508004B80401C8028FCDB2046611ECCB20028D6D10A
S31508004B9000BF00F091F900F007F800BFC0E7000079
S31508004BA014020020FBAA000010B57E20FFF79AFB2E
S31508004BB0FDF7E8FF0B490C4881820F211430FFF7F7
S31508004BC059FC09491431C883802107481430FDF778
S31508004BD073FF7E20FFF786FB802103481430FDF71C
S31508004BE077FF10BDFBAA00000002002070B504463E
S31508004BF000257E20FFF776FB98480088FA280ADD0C
S31508004C0000209649088096490870FF21013193488B
S31508004C10801DFCF7C2FE924800780300FFF7C9FB27
S31508004C2008052031425BD5ECFDFC7E2C11D1002015
S31508004C308A49088001208A490870884801880088BE
S31508004C40401C864A1080901D445400201146C870A6
S31508004C5002E0002081490880002080490871FBE0B5
S31508004C607E4801880088401C7C4A1080901D445468
S31508004C7002207B4908701046007900191146087110
S31508004C80EAE0764801880088401C744A1080901D26
S31508004C9044540320724908701046007900191146D9
S31508004CA00871D9E06D4801880088401C6B4A10805D
S31508004CB0901D445404206A4908701046007900196A
S31508004CC0114608710846C470C078002802D105202C
S31508004CD063490870C0E061484079012856D15E2CC6
S31508004CE01CD15E4800797E305C4908717E215B489C
S31508004CF002880088401C594B1880981D8154801FD3
S31508004D00C078401EC0B21946C870002802DC0520CB
S31508004D105349087000205149487155E05D2C1CD153
S31508004D204E4800797D304D4908717D214B480288EF
S31508004D300088401C494B1880981D8154801FC078F4
S31508004D40401EC0B21946C870002802DC0520444936
S31508004D50087000204149487136E04048007900193A
S31508004D603E490871084601880088401C3B4A108065
S31508004D70901D4454801FC078401EC0B21146C870AA
S31508004D80002821DC0520364908701DE07D2C03D15A
S31508004D9001203249487117E03048007900192F4937
S31508004DA00871084601880088401C2C4A1080901D0E
S31508004DB04454801FC078401EC0B21146C8700028EF
S31508004DC002DC05202649087046E024480079C043DD
S31508004DD0401CC5B2A54203D106202149087002E04D
S31508004DE007201F4908701D4801880088401C1B4A77
S31508004DF01080901D44542FE0184801880088401CF4
S31508004E00164A1080901D44547E2C0BD1012115485A
S31508004E1001720020114601E01DE00DE008801049EE
S31508004E20087008E000200D49088000210D4801722D
S31508004E3000200B4908700FE0002009490870074850
S31508004E4001880088401C054A1080901D44540020A3
S31508004E501146088000E000BF00BF70BDF8040020BE
S31508004E60B7010020A003002070B5024600201346B3
S31508004E700C461D02FF26360235402543284670BDDE
S31508004E8000BF00BF00BF00BF00BF00BF00BF00BF1C
S31508004E9000BFFEE706490748818200211430418099
S31508004EA05F218180C1800181002141817047000016
S31508004EB0FBAA00000003002000B5134913488182AD
S31508004EC0FF21143041800F210181A021C180D22108
S31508004ED081801E214181AF21C1818C210182BE21A1
S31508004EE081810B4901830A49233141830521418286
S31508004EF00A218182C182002181830F21FFF7BAFA34
S31508004F0002491431C88300BDFBAA00000002002034
S31508004F105A25000010B57E20FFF7E4F95648C07AF6
S31508004F2001282AD15448407A01281CD15349486897
S31508004F30C821FCF7EFFCC007C00F002805D1802167
S31508004F400920C006FDF7AFFF0DE04C494868C821A7
S31508004F50FCF7E0FCC007C00F002804D08021092018
S31508004F60C006FDF7A2FF10210920C006FDF79BFF2A
S31508004F7001214348FDF797FF10BD3F48407A0128B5
S31508004F8078D13D482030007A002802D0012834D153
S31508004F900BE040213A48FDF77DFF002802D1FEF7D5
S31508004FA0C7FF01E0FFF72CF863E034494868FF21A2
S31508004FB0F531FCF7AFFCC007C00F00280ED18021E1
S31508004FC00920C006FDF771FF01212D48FDF76DFF89
S31508004FD010210920C006FDF768FF0DE08021092091
S31508004FE0C006FDF760FF10210920C006FDF75BFF2C
S31508004FF001212348FDF757FF3BE01F482030007A80
S31508005000052827D11D494868FF21F531FCF782FCA0
S31508005010C007C00F00280ED180210920C006FDF761
S3150800502044FF01211648FDF740FF10210920C0065C
S31508005030FDF73BFF1CE080210920C006FDF733FF82
S3150800504010210920C006FDF72EFF01210C48FDF7A7
S315080050502AFF0DE080210920C006FDF726FF012161
S315080050600748FDF722FF10210920C006FDF71DFF9E
S3150800507000BF00BF00BF7FE7A0030020C0010020DB
S3150800508000040048FEF75AFCFEF77EF9FDF712FC0D
S31508005090FDF7AEF90B20FDF7DDF80C20FDF7DAF881
S315080050A00920FDF7D7F80320FDF7D4F80121564863
S315080050B0FDF744FA4B200002FDF766FBFEF7A2F85F
S315080050C0FEF772FC0D216320FEF79CFC01214F4878
S315080050D041720021C172FFF705FDFEF7DFFD00F002
S315080050E09DF8FEF725FF7F217E20FFF739F98AE034
S315080050F04648C07900280AD1FDF748FAFFF70AFFA3
S31508005100FFF7CCF9FEF7B2F800F07AFF78E03F48EF
S31508005110C079012836D1002301221946184600F025
S31508005120A9F900231A461946184600F0A3F9384883
S3150800513040683849884204D908213748FDF7B3FE44
S315080051401DE033494868FF21F531FCF7E3FBC0074A
S31508005150C00F00280ED180210920C006FDF7A3FE46
S3150800516010210920C006FDF79EFE01212A48FDF7F9
S315080051709AFE04E010210920C006FDF796FEFDF709
S31508005180AFFA3DE02148C079022839D1FDF7FEF98A
S31508005190FEF76CF8002301221946184600F06AF952
S315080051A000231A461946184600F064F9184840685C
S315080051B01849884204D908211748FDF774FE1DE0EE
S315080051C013494868FF21F531FCF7A4FBC007C00F57
S315080051D000280ED180210920C006FDF764FE1021A3
S315080051E00920C006FDF75FFE01210B48FDF75BFEAF
S315080051F004E010210920C006FDF757FEFFF78EFBD5
S315080052007E20FFF76FF873E700240140A003002013
S31508005210C0010020204E00000004004810B54021BF
S315080052200F48FCF7BAFB40210D48FDF727FC06217D
S315080052300B48FFF71FF90A49898988420AD10848A5
S315080052401438808A0749884208D0FFF723FEFFF7FB
S3150800525069F803E0FFF71EFEFFF764F810BD0000CB
S3150800526014030020FBAA0000F7B5A0B00C461546AB
S3150800527080216846FCF791FB002700267E216846B8
S315080052800170FE214170EF2181700721C1702099BC
S3150800529001710021417184712112C17101210172CC
S315080052A0457229128172012605E06846805DC0199B
S315080052B0C7B2701CC6B20B2EF7DBF843401CC1B24E
S315080052C06846C1727E2101730D21FEF753FD23B096
S315080052D0F0BDFFB585B005460E460E9F002001902D
S315080052E0029003900490009000247E216846017184
S315080052F0457186710421C171079901720899417235
S3150800530087723912C172012407E001A8015D00986D
S315080053100818C0B20090601CC4B2082CF5DB0098CF
S31508005320C043401CC1B2684601737E2141730A21FD
S3150800533001A8FEF71FFD09B0F0BDF7B584B0054614
S315080053400E4600200090019002900390002700244A
S315080053507E2168460170467085700121C1706946D4
S3150800536006980871012405E06846005DC019C7B2B1
S31508005370601CC4B2052CF7DBF843401CC1B2684672
S3150800538041717E2181710721FEF7F4FC07B0F0BD5B
S3150800539070B504460D467E20FEF7A4FF03E020788C
S315080053A0641CFEF7D7FC2846691E8DB20028F6D184
S315080053B070BD000030B5A1B00446802101A8FCF7F5
S315080053C0ECFA0025002C02D0012C20D10FE07E211A
S315080053D06846017100214171442181711321C1710F
S315080053E01522104902A8FCF7BFFA192510E07E21FC
S315080053F068460171FE214171442181713321C171D1
S315080054003622094902A8FCF7AFFA3A2500E000BFA0
S3150800541000BF802D03DA294601A8FFF7B9FF21B09E
S3150800542030BD00006C01002081010020F8B5064659
S315080054300C46FCF7ABFE051E0F4600D001200143C3
S3150800544049000B484908411AC90F0DD0002E01D052
S31508005450012100E000210C4361004908401AC00FF1
S3150800546002D10120FFF700F828463946F8BD0000AA
S315080054700000F07FFFB58DB005460E4617460020A2
S315080054800B9000240A9009900890FE48007864283A
S3150800549003D0FD48C078642804D10121FA48203891
S315080054A0017303E00021F84820380173002F02D069
S315080054B0012F7BD130E2F548C089B04202D1F348CA
S315080054C0C48A00E00524052C01DC052402E0322C00
S315080054D000DB0524301BA8420FDDEB482038C07BD3
S315080054E000284CD1E94854384068E849543988615D
S315080054F00121E5482038C17341E03019A8423EDC55
S31508005500E1482038C07B012839D1DF484079012895
S315080055102FD1DE4854384068DC4954398969401A25
S31508005520DB4988420DD2D848AC380089462820DDA8
S31508005530D548AC380089801E81B2D348AC38018181
S3150800554017E0D24854384068D04954398969401A16
S315080055507D21890188420CD9CB48AC3800895F285F
S3150800556007DAC948AC380089801C81B2C648AC380D
S3150800557001810121C448417100212038C173C24804
S315080055802038C07B012878D1301BA84276DDBF4879
S31508005590543840687D21C900884208D26420B94938
S315080055A008700021B84820388174AEE1FEE3B64899
S315080055B02038807C00286AD10121B34820388174BC
S315080055C0B248808964285ADAAF484038818AC08B45
S315080055D0081A81B2AC48403801840146088CFCF7A9
S315080055E058FC01460690AB480068FCF777FA079026
S315080055F0FCF7AAFCA84A03C2A3494039898C494347
S315080056000846FCF74DFC07910690A3480CC8069877
S31508005610FCF754FBA04A03C29F4903C9FFF706FFDC
S3150800562007910690FCF7B8FC9C49086096494039F2
S31508005630888CFCF72EFC0146059098480068FCF714
S315080056404DFA97490690FCF70CFA0790FCF74AFCC6
S31508005650944908700846007864280ADC8D48006872
S31508005660FCF772FC0022904B07910690FCF780FC31
S3150800567008D864208B49087004E043E15BE06420A5
S315080056808849087080484038818A41873DE17F48CB
S315080056905438406C7D21C900884247D900207B498F
S315080056A0543948647F48007864283BDA764840389D
S315080056B0818A408F814230DD01218907754800685B
S315080056C0FCF776F90790FCF70DFC81B26E48403876
S315080056D0828A408F101A814205DA72480078801E45
S315080056E0704908701EE0684940398A8A498F501AFD
S315080056F0FCF7C4FB0790674801680798FCF768FC45
S3150800570010D268480078801C6649087008460078F8
S31508005710642807DD6420087004E062480078401DAC
S315080057206049087058484038818A41875D48007842
S3150800573054490870E9E054484079002870D1534824
S315080057408089642803DB64204E490870DDE04F48F1
S31508005750543840687D21C900884207D264204949E7
S3150800576008700021484820388174CEE04648203821
S31508005770807C00285DD10121434820388174434844
S31508005780808964284DDA40484038818AC08B081AD7
S3150800579081B23D48403801840146088CFCF779FB04
S315080057A0014606903B480068FCF798F90790FCF715
S315080057B0CBFB394A03C234494039898C49430846E8
S315080057C0FCF76EFB0791069033480CC80698FCF761
S315080057D075FA314A03C2304903C9FFF727FE079114
S315080057E00690FCF7D9FB2D49086027494039888C73
S315080057F0FCF74FFB0146059028480068FCF76EF950
S3150800580027490690FCF72DF90790FCF76BFB25490D
S31508005810087008460078642806DD6420087003E0EE
S315080058206AE064201F49087017484038818A418712
S315080058306BE016485438406C7D21C900884256D919
S3150800584000201249543948640F484038818A408FED
S31508005850814244DD012189070E480068FCF7A8F853
S315080058600790FCF73FFB81B207484038828A408F91
S31508005870101A81421ADA0B480078801E0949087006
S3150800588032E00000EA000020C003002014020020D5
S3150800589070170000CC000020D0000020D80000209F
S315080058A00000C842E90000200000F03FFE498A8A4D
S315080058B0498F501AFCF7E2FA0790FC4801680798E6
S315080058C0FCF786FB10D2FA480078801CF849087065
S315080058D008460078642807DD6420087004E0F44868
S315080058E00078401DF2490870EF48818A4187F048E0
S315080058F00078F049087008E0EB486C38007AED4902
S31508005900087002E00020EB490870EA480278384639
S315080059101099FFF78DF862E3E3484030007A0128D2
S3150800592004D002287DD003287CD196E0E24840883E
S31508005930B04202D1E048448A00E00A24DE484188A1
S31508005940408A081AA84209DBDB4854384068DA4915
S31508005950543988620020D94908701AE0D648408828
S31508005960A84216DCD5480078002812D1CE48818C8A
S3150800597081870120D1490870CF4854384068CE49FC
S315080059805439896A401ACC4954390862084640682D
S315080059900863C9488188808A081AA84209DB00205A
S315080059A0C7490870C44854384068C3495439C8625E
S315080059B017E0C1488088A84213DCC148007800284F
S315080059C00FD1B948818CC1870120BD490870BA48F2
S315080059D054384068B8495439C96A401AB6495439DE
S315080059E04862B548543840687D21C90088422AD3A0
S315080059F0AD482030407C002825D1AB48818C40300A
S31508005A000180012120384174014620310888FCF7BD
S31508005A1040FA01460590AB48FCF760F8AA4906909B
S31508005A2001E011E022E0FCF71CF80790FCF75AFAAF
S31508005A30C1B29D48403001710079642803DB6421B6
S31508005A409948403001711AE09B484088B04202D11B
S31508005A509948448A00E00A2411E097488088B042B1
S31508005A6002D19548848A00E00A2408E09248808892
S31508005A70B04202D19048848A00E00A2400BF00BFE1
S31508005A80052C01DC052402E0322C00DB3224301B15
S31508005A90A8421ADB88485438406887495439C8618F
S31508005AA0002048638863804845842030007C0028AD
S31508005AB006D11E217C4840308170012120380174AE
S31508005AC0002179482030417312E13019A84211DCCF
S31508005AD075482030007C0128F6D100217248203014
S31508005AE00174FF38E138406873495439C8610020A9
S31508005AF04863FDE0B542E7DB6B484030007A012891
S31508005B00E2D16948403080790028DDD16A48408A68
S31508005B100A280BDB68495439086AFCF7BAF96B4955
S31508005B200790FBF7DBFF6A4908601EE06248408A77
S31508005B300A280FDA6048408A07280BDD5E4954397F
S31508005B40086AFCF7A6F963490790FBF7C7FF60499F
S31508005B5008600AE058495439086AFCF79AF95E4918
S31508005B600790FBF7BBFF5A4908604F49888FFCF737
S31508005B7090F94D490690888FFCF78BF904905448A4
S31508005B8001680498FBF76DFF05900699FBF769FF16
S31508005B900790FCF7D9F9514A03C24349888FFCF7A5
S31508005BA093F9039102904D4903C9FFF73FFC019110
S31508005BB00090039B029AFCF7E9F80022484B0591EE
S31508005BC00490FCF77BF807910690FCF79FF981B2E1
S31508005BD035486C38818038495439486AFCF759F990
S31508005BE03C490790FBF77AFF394908602E49C88F68
S31508005BF0FCF74FF92C490690C88FFCF74AF9049030
S31508005C00334801680498FBF72CFF05900699FBF7C3
S31508005C1028FF0790FCF798F9304A03C22249C88F33
S31508005C20FCF752F9039102902C4903C9FFF7FEFBD2
S31508005C3001910090039B029AFCF7A8F80022284BD2
S31508005C4005910490FCF73AF807910690FCF75EF97F
S31508005C5081B215486C38C18017488089642844DAAF
S31508005C6015498889FCF715F9134954390690086BC4
S31508005C70FCF70FF91B490290FBF730FF0E49049019
S31508005C804A880949898B501AFCF7F8F80390049951
S31508005C90FBF724FF05900699FBF7E3FE0A490790F0
S31508005CA0FBF71CFF01491FE080030020CC00002001
S31508005CB0E9000020EA00002014020020DC00002091
S31508005CC0DD000020000082430000C84200803B45FA
S31508005CD0C40000200000FA440080BB44E000002015
S31508005CE00000594000007A4408600121BE488171CD
S31508005CF0BD482038007C00287CD001287BD1BA48D2
S31508005D008078BA490978884208DA0021B64881704D
S31508005D10203801740020B64988641CE1301BA8426B
S31508005D2010DDB1482038407C012803D1AE480179FE
S31508005D30C17002E06421AC48C1700121AA4820382C
S31508005D40017308E1A848007A012804D0022813D074
S31508005D5003287DD188E03019401BA04208DA3019A3
S31508005D60401B201A5F21081AC1B29F48C17002E081
S31508005D705F219D48C170EDE09D48406B9C49896B49
S31508005D80401A7D21C90088424BD99948406B9849E9
S31508005D90886395484038408CA84211DD9248AC3853
S31508005DA080880A3081B29048AC3800E017E18180DB
S31508005DB0C088642832DB64218B48AC38C1802DE06A
S31508005DC089494039498C691AE20F12195210521C36
S31508005DD0914211DA8448AC388088801C81B28248A6
S31508005DE0AC388180C088642818DB64217E48AC38CA
S31508005DF0C18013E0B0E0DBE07B494039498C691A81
S31508005E00E20F12195210921C914207DD7648AC38FF
S31508005E108088801E81B27448AC38818072484038C8
S31508005E204584734840687249C969401A714988426D
S31508005E3014DD6D48AC388088401D81B26A48AC389C
S31508005E4081808088642805DB64216748AC3800E0D7
S31508005E507CE08180664840686549C8616248AC381C
S31508005E600179AC30C17075E06148406B6049896B57
S31508005E70401A7D21C900884247D95D48406B5C4974
S31508005E80886359484038408CA8420FDD5648AC38DC
S31508005E90C0880A3081B25448AC38C180C0886428AA
S31508005EA030DB64215048AC38C1802BE04E4940397C
S31508005EB0498C691AE20F12195210521C91420FDAD4
S31508005EC04948AC38C088801C81B24748AC38C18084
S31508005ED0C088642816DB64214348AC38C18011E0C9
S31508005EE041494039498C691AE20F12195210921C1D
S31508005EF0914207DD3C48AC38C088801E81B23A48DA
S31508005F00AC38C180384840384584394840683849F3
S31508005F10C969401A3849884212DD3348AC38C08806
S31508005F20401D81B23048AC38C180C088642803DB84
S31508005F3064212D48AC38C1802D4840682C49C86179
S31508005F402948AC388179AC30C17003E03221264843
S31508005F50C17000BF00BF2FE02348007A012823D173
S31508005F603019A8421CDB2048AC380179AC30C17026
S31508005F703019801EA8420FDD20480078002816D167
S31508005F801948AC388088401D81B21748AC388180E2
S31508005F9001201A4908700AE000201849087006E02E
S31508005FA000211148C17002E00A210F48C17003E0C0
S31508005FB000210D48C17000BF00BF0B48007A0128B8
S31508005FC006D10948C27838461099FEF731FD05E032
S31508005FD00548827838461099FEF72AFD00BF00BFAB
S31508005FE00B9811B0F0BD0000C0030020EA000020A5
S31508005FF0C001002088130000581B0000E80000209C
S3150800600010B5FA48007A002872D0F8484038C08A95
S31508006010FF217D31884204DCF4484038808A884272
S315080060200ADDF2482038C07A002805D1F0494860D0
S315080060300121EE482038C172ED48C06BED4988420F
S315080060400AD9EA482038C07A002805D1E8494860C4
S315080060500121E6482038C172E4482038C07B01286F
S315080060601ED1E348C06CE44988421DD90020E049A6
S31508006070C864DE484038418B808A81420BDBDB48A6
S315080060802038C07A00280FD1D94948600121D7485D
S315080060902038C17208E0D5484038818A418303E038
S315080060A0D2484038818A4183D0482038007C01286C
S315080060B01FD1CF48806CD04988421ED90020CC49D0
S315080060C08864CA484038018BC08A81420BDBC748BE
S315080060D02038C07A002810D1C54948600121C34834
S315080060E02038C17209E0C1484038C18A018304E0FA
S315080060F036E0BE484038C18A0183BC482038C07A99
S3150800610001282DD1B9482038407A012828D1002302
S31508006110012219461846FFF7ADF900231A46194613
S315080061201846FFF7A7F9B24840687D210901884259
S3150800613015D90020AE49486010210920C006FCF791
S31508006140B2FE80210920C006FCF7ADFE0121AB484E
S31508006150FCF7A9FE0021A54820384172C17210BD7E
S31508006160A2482038407A002863D110210920C006A9
S31508006170FCF799FE80210920C006FCF794FE012150
S315080061809E48FCF790FE00219848017200230122E0
S3150800619019461846FFF76EF900231A461946184697
S315080061A0FFF768F992484068FF21F531884204D222
S315080061B020219248FCF779FE4BE220218F48FCF714
S315080061C072FE8B4840688C498842F5D98748203842
S315080061D0807B002817D1864840687D21490188427E
S315080061E001D2FDF769FE08218448FCF75CFE002110
S315080061F07E482038C17220304171817100207C4967
S31508006200086208630BE040217C48FCF743FE00283F
S3150800621005D00021754801720121203841722021DC
S315080062200920C006FCF73FFE7D2040017049486002
S315080062300FE26E48007A0300FEF7BBF8060472CD3B
S31508006240FEFDFC7100216948417181710020684991
S31508006250086208630023012219461846FFF70AF95F
S3150800626000231A4619461846FFF704F95F484038CE
S31508006270C18A81832030C079012809D15C48006928
S315080062805F49884203D9002158482038C17166E71A
S31508006290574840687D210901884228D9002153487A
S315080062A0C17100205249486040215448FCF7F2FD6C
S315080062B0002809D1FDF700FE08215048FCF7F3FD38
S315080062C0FF20F530FCF7B8FA10210920C006FCF7C4
S315080062D0EAFD80210920C006FCF7E5FD01214748B3
S315080062E0FCF7E1FD20214548FCF7DDFD17E02021FC
S315080062F00920C006FCF7D9FD08214048FCF7D5FD62
S315080063003B484068FF21F531884208D93748AC3800
S315080063104089002803D120213848FCF7C4FD97E1BD
S3150800632033484068FF21F531884204D2202133489A
S31508006330FCF7BBFD03E020213048FCF7B4FD2C49EF
S3150800634048687D21C900FBF7E5FA232823D22849A6
S3150800635048687D21C900FBF7DDFA19281BD92348AF
S315080063604038818AFF386D384088814207DA1F48ED
S315080063704038C18AFF386D38408881421ADB1B488D
S315080063808079012816D1002019494860C861022180
S31508006390164801720EE0164948687D21C900FBF7C8
S315080063A0B9FA232806D3002011494860C86102219A
S315080063B00E4801720E4A54325188FF326D32D08A25
S315080063C001231A46FFF756F800231A4619461846B7
S315080063D0FFF750F83CE106484068FF21F53188424E
S315080063E010D220210548FCF760FD0FE0C00300200D
S315080063F0C001002070110100B80B0000000400481D
S315080064008813000020219548FCF74DFD9448416803
S31508006410543000897D22D2005043814214D2904ADA
S3150800642054325188FF326D32D08A01231A46FFF75B
S3150800643021F802E09AE057E013E000231A461946CD
S315080064401846FFF717F80BE000218648017400206C
S315080064508349486001218348417303212030017232
S31508006460F6E080482038C08AFF217D31884204DC66
S315080064707C482038808A88420CDD00230122194690
S315080064801846FEF7F7FF00231A4619461846FEF780
S31508006490F1FF28E0724948687D21C900FBF73AFAFE
S315080064A06F4954314989884210D26D4A54329188CD
S315080064B0FF326D32D08A01231A46FEF7DBFF00232E
S315080064C01A4619461846FEF7D5FF0CE065482038E7
S315080064D0818AC183002062494860002161480174AD
S315080064E0042120300172B3E05E482038C08AFF21BB
S315080064F07D31884204DC5B482038808A88420CDD7E
S315080065000023012219461846FEF7B4FF00231A464F
S3150800651019461846FEF7AEFF27E0514948687D211F
S31508006520C900FBF7F7F94E495431098A0F398842F1
S3150800653014D24B4A5432D189FF326D32908A0123E4
S315080065400022FEF797FF464A5432D188FF326D3251
S31508006550D08A01231A46FEF78DFF06E0002040493F
S31508006560486005213F482030017271E03C48406888
S31508006570FF21F531884204D220213848FCF795FCE2
S315080065800FE037484068FF21F531884209D9344879
S3150800659040684B21C900884203D220212F48FCF7C6
S315080065A082FC2F484068304988422DD22D48203831
S315080065B0C08AFF217D31884204DC2A482038808A37
S315080065C088420CDD0023012219461846FEF752FFC1
S315080065D000231A4619461846FEF74CFF37E0204AAC
S315080065E05432D189FF326D32908A01230022FEF798
S315080065F041FF1B4A5432D188FF326D32D08A0123BB
S315080066001A46FEF737FF22E020211448FCF74DFC16
S31508006610134840681449C831884218D300201049E5
S31508006620486000210F48203001722038417200234B
S31508006630012219461846FEF71DFF00231A46194679
S315080066401846FEF717FF20210448FCF72CFC00BF6C
S3150800665000BF7E20FDF746FE00BF80E50004004827
S31508006660C0010020A0030020A43800008C660008A2
S31508006670C000002000010000484400088C6700089C
S31508006680C00100204008000058440008000000002F
S3150800669000000000000000000000000000000000EC
S315080066A000000000000000000000000000000000DC
S315080066B000000000000000000000000000000102C9
S315080066C003040102030406070809000000A24A049D
S315080066D00000000000000000010203040607080984
S315080066E0000000000000000000000000000000009C
S315080066F00400000001000000000000000000000087
S31508006700000000000000000000000000000000007B
S31508006710000000000000000000000000000000006B
S31508006720000000000000000000000000000000005B
S31508006730000000000000000000011058594C4C30C1
S315080067403131327878787878787878CB7E0001108D
S3150800675058594C4C3031313278787878787878785E
S3150800676004013205054C4C3031310614594132309A
S31508006770303532384834353034324178787878785C
S311080067807D5D7E000000000000000000A7
S705080018C515
